:100000001DC02CC02BC02AC029C028C027C026C0B4
:1000100025C024C023C022C021C020C01FC01EC0D4
:100020001DC01CC01BC01AC019C018C017C016C004
:1000300015C014C013C012C011C010C011241FBEBF
:10004000CFEFD1E0DEBFCDBF21E0A0E0B1E001C045
:100050001D92A031B207E1F702D002C0D1CF50D635
:04006000F894FFCF42
:100D000011241FBECFEFD1E0DEBFCDBF21E0A0E0B8
:100D1000B1E001C01D92A031B207E1F7F894BA9A90
:100D200088ED8093710081E080937300E7EEFFE02F
:100D3000949090927400809180001092860010929E
:100D400085001092840010928300D2981092820045
:100D500023E0209381001092860080E1809385003B
:100D600096E09093840010928300809165008E7FBE
:100D700080936500D59A1092920020939100109272
:100D8000960088E0809395009093940010929300D1
:100D900040E060E280E2E1D0AA24AA94C0E8809119
:100DA000860087FFFCCF80918000882E8093900082
:100DB000982F92959F70692E8F70782E912C10C06D
:100DC0008091860087FFFCCF2091800020939000C7
:100DD000892DE92DF0E0E050FF4F20838F5F982EA2
:100DE000991670F3872D8B3099F018F4823041F00A
:100DF000D6CF8C3009F439C08D3009F466C0CFCF1E
:100E0000409103016091020180910101A6D0C7CFFA
:100E1000953029F6309100013D3008F6209101010E
:100E2000822F8F7309F0BBCF80910401803509F0C8
:100E3000B6CF29018091020190E0830F911D8F3F71
:100E4000910509F0ACCF8091030190E0820F911DD4
:100E50008F3F910509F0A3CFF20113E017BFE8958A
:100E600017B710FDFDCFA12C9ACF983009F097CF7E
:100E700087E08A1508F493CF40E06FEF80E06DD0F3
:100E80000F921F9224E0A0E0B1E011E0F2010D907A
:100E90001D9017BFE895EE5F2A95C9F7A394A0FCB3
:100EA00008C015E0F201E07F17BFE89517B710FD05
:100EB000FDCF1F900F909AE49A95F1F740E060E023
:100EC0008A2D4BD088E0480E6ACF933009F067CF67
:100ED000809100018F3F09F062CF8091860087FFEB
:100EE000FCCF80918000882E9091960095FFFCCFDA
:100EF000809390008D3109F052CF8091860087FF5A
:100F0000FCCF80918000882E9091960095FFFCCFB9
:100F10009FEF980F90939000811141CF8091010134
:100F200090E0982F882720910201822B2091960033
:100F300025FFFCCFC0939000912C0BC03091960000
:100F400035FFFCCFFC01E20FF11DE491E09390002E
:100F50009394292D283090F322CFBA9A4F936F9310
:100F60008F9343E05F9168E057FF06C032E0C29A7A
:100F70003A95F1F7C29805C0C29AC29832E03A9504
:0E0F8000F1F7550F6A9581F74A9561F70895CC
:100FD0005BBA920959E0436EF3F4C816B6938D21BB
:080FE0008005637595B5BF9D06
:00000001FF
